:1000000019C033C032C031C030C02FC02EC02DC087
:100010002CC02BC02AC029C028C027C066C1B6C1C9
:1000200024C023C022C021C020C01FC01EC01DC0CC
:100030001CC01BC011241FBECFEFD2E0DEBFCDBF5E
:1000400011E0A0E0B1E0E0E7F8E002C005900D9219
:10005000AC30B107D9F721E0ACE0B1E001C01D92AE
:10006000A331B207E1F7EAD101C4CACF55B121E00B
:1000700030E0B90102C0660F771F8A95E2F7CB0125
:10008000462F4095542355B924B1262B24B920EE90
:1000900031E072E07A95F1F700C021503109211565
:1000A0003105B9F724B1422344B92CE330E042E0F2
:1000B0004A95F1F700C02150310921153105B9F7F2
:1000C00093B1892324EA31E052E05A95F1F700C058
:1000D0002150310921153105B9F7089545B121E0C5
:1000E00030E0F90102C0EE0FFF1F8A95E2F7CF0161
:1000F0002E2F2095422345B994B1892B84B9F2E083
:10010000FA95F1F700C0662379F084B1822384B9AF
:100110000BC032E03A95F1F700C001970097C9F79C
:1001200084B1282324B908958CE390E0F2CF45B13F
:1001300021E030E0082E02C0220F331F0A94E2F7BC
:10014000922F9095392F342335B934B1232B24B90C
:1001500022E02A95F1F700C024B1922394B928E057
:1001600030E042E04A95F1F700C0215031092115F5
:100170003105B9F723B130E0A90102C05595479583
:100180008A95E2F7CA0181702DE230E052E05A957B
:10019000F1F700C02150310921153105B9F7089553
:1001A0001F93CF93DF93182FC8E0D0E0812FBFDFDC
:1001B00020E8829FC0011124D695D82BC150B1F7F9
:1001C0008D2FDF91CF911F9108951F93CF93DF93D0
:1001D000182FD62FC8E06D2F6170812F7FDFD69545
:1001E000C150C9F7DF91CF911F910895CF93C82FC8
:1001F0003DDF6CEC8C2FE9DF64E48C2FE6DFCF91E0
:1002000008951F93CF93DF93C82F30DF6CEC8C2FB2
:10021000DCDF6EEB8C2FD9DF8C2FC2DF182F8C2FF9
:10022000BFDFD82F8C2F22DF612F70E07D2B882736
:1002300077FD8095982F04D220E030E040E25FE324
:100240008BD2CBD1633E24E0720714F062EE74E0EF
:10025000CB016A3D2DEF720714F48AED9DEFDF911B
:10026000CF911F910895882341F0EFE1FEE431978B
:10027000F1F700C000008150C1F708951BB88FEF5F
:100280008AB988B1807F88B987B18F6087B9209893
:10029000289A82E084BD84E085BD83E387BD86E043
:1002A00080936E0080E480937C0087E880937A00DE
:1002B00010920C011092110110921201789408957D
:1002C000ECE7F0E090819C7F90839081892B808384
:1002D000EAE7F0E0808180648083808186FDFDCF45
:1002E000809178009091790008951F920F920FB637
:1002F0000F9211242F933F934F936F937F938F937C
:100300009F93EF93FF931BB888B18F6088B9E091FA
:100310000C01F0E0E35FFE4FE081F0E0E050FF4FC2
:1003200080818BB98091110120910C0190E002C075
:10033000959587952A95E2F780FD5F9A48B180915F
:100340000C0121E030E0B90102C0660F771F8A95E9
:10035000E2F7CB018095842388B980910C018F5FEF
:1003600080930C0180910C01843010F010920C01EC
:10037000FF91EF919F918F917F916F914F913F915D
:100380002F910F900FBE0F901F9018951F920F92F4
:100390000FB60F9211248F931BB888B18F6088B964
:1003A0008F910F900FBE0F901F901895CF93DF93F2
:1003B0009C01273E83E0380791F133233CF43195CB
:1003C00021953109E22F432FDAE011C0C90168EE0F
:1003D00073E025D2E82F492F283E83E0380734F018
:1003E000C90168EE73E01BD2D62F01C0DBE08E2F6F
:1003F000942F64E670E013D26AE070E010D2C62F4A
:10040000F82F2436310534F08E2F942F64E670E0F7
:1004100006D201C06BE084E08093110104C06AE061
:10042000CAE0FAE0DAE0D0930D0160930E01C093C8
:100430000F01F0931001DF91CF9108951FDF87EE38
:1004400093E0B4DF10E06894FF24F1F803E0CFEF0D
:10045000D0E0E12C01C01F2D113051F028F01230F6
:1004600061F0133019F1F8CF81E0C0DE11E0F4CF74
:1004700081E05DDE8111EFCFEFCF81E0C2DE189920
:1004800012C0BC01882777FD8095982FD9D026E629
:1004900036E646EE5FE360D120E030E040EA53E428
:1004A00038D09BD0CB0182DF102FD6CF89E1DBDEA5
:1004B00085E006DF209112019695879596958795A0
:1004C000AE01481B590BCA01969587959927820F53
:1004D000911D95958795809312012091120187B502
:1004E00030E090E003978217930724F487B5835098
:1004F0008093120180911201853018F485E0809379
:10050000120187B590911201891B88BD1E2DA4CFC1
:100510005058BB27AA270ED0E5C0D6D030F0DBD08C
:1005200020F031F49F3F11F41EF4CBC00EF4E0959F
:10053000E7FBC1C0E92FE7D080F3BA176207730762
:100540008407950718F071F49EF5FFC00EF4E0954E
:100550000B2EBA2FA02D0B01B90190010C01CA017D
:10056000A0011124FF27591B99F0593F50F4503E28
:1005700068F11A16F040A22F232F342F4427585F1A
:10058000F3CF469537952795A795F0405395C9F732
:100590007EF41F16BA0B620B730B840BBAF09150EA
:1005A000A1F0FF0FBB1F661F771F881FC2F70EC089
:1005B000BA0F621F731F841F48F48795779567955C
:1005C000B795F7959E3F08F0B3CF9395880F08F045
:1005D0009927EE0F97958795089504D06894B111E7
:1005E000B5C0089598D088F09F5790F0B92F9927FB
:1005F000B751A0F0D1F0660F771F881F991F1AF02E
:10060000BA95C9F712C0B13081F09FD0B1E008951A
:100610009CC0672F782F8827B85F39F0B93FCCF39B
:10062000869577956795B395D9F73EF49095809523
:10063000709561957F4F8F4F9F4F0895E89409C043
:1006400097FB3EF490958095709561957F4F8F4F05
:100650009F4F9923A9F0F92F96E9BB279395F6951B
:10066000879577956795B795F111F8CFFAF4BB0F99
:1006700011F460FF1BC06F5F7F4F8F4F9F4F16C0FD
:10068000882311F096E911C0772321F09EE8872F87
:10069000762F05C0662371F096E8862F70E060E043
:1006A0002AF09A95660F771F881FDAF7880F9695BC
:1006B000879597F9089597F99F6780E870E060E063
:1006C00008959FEF80EC089500240A9416161706EB
:1006D00018060906089500240A9412161306140633
:1006E00005060895092E0394000C11F4882352F096
:1006F000BB0F40F4BF2B11F460FF04C06F5F7F4F4E
:100700008F4F9F4F089557FD9058440F551F59F034
:100710005F3F71F04795880F97FB991F61F09F3FEE
:1007200079F087950895121613061406551FF2CF17
:100730004695F1DF08C0161617061806991FF1CF67
:1007400086957105610508940895E894BB2766278E
:100750007727CB0197F908950BD0C4CFB5DF28F0E8
:10076000BADF18F0952309F0A6CFABCF1124EECF56
:10077000CADFA0F3959FD1F3950F50E0551F629FFC
:10078000F001729FBB27F00DB11D639FAA27F00DEA
:10079000B11DAA1F649F6627B00DA11D661F829F11
:1007A0002227B00DA11D621F739FB00DA11D621FF6
:1007B000839FA00D611D221F749F3327A00D611D13
:1007C000231F849F600D211D822F762F6A2F1124F5
:1007D0009F5750408AF0E1F088234AF0EE0FFF1F48
:1007E000BB1F661F771F881F91505040A9F79E3F7F
:1007F000510570F060CFAACF5F3FECF3983EDCF379
:10080000869577956795B795F795E7959F5FC1F7BB
:10081000FE2B880F911D9695879597F9089597FB64
:10082000072E16F4009406D077FD08D00BD007FCF5
:1008300005D03EF4909581959F4F089570956195F0
:100840007F4F0895AA1BBB1B51E107C0AA1FBB1F06
:10085000A617B70710F0A61BB70B881F991F5A954C
:10086000A9F780959095BC01CD010895F894FFCF2C
:0C0870003F065B4F666D7D077F6F400008
:00000001FF
